:03000000020246B3
:10000300C000784AD8FED00022C000C001790A7827
:10001300B8D8FED9FADAF6D001D00022D2B1120054
:1000230003C2B112000322A2E792A3A2E692A2A204
:10003300E592A1A2E492A012001FA2E392A3A2E27E
:1000430092A2A2E192A1A2E092A012001F22D28763
:1000530002002AC28702002AC2B1C2B0C0027A28B3
:1000630012000CD00274331200567433120056740B
:10007300321200567428120056740C120056740182
:10008300120056C0027A0212000CD00222E49360DE
:1000930006120051A380F62244404480020056C059
:1000A300E0E8C4540F4430120051E8540F443012B6
:1000B3000051D0E02210990280FBF599221098029A
:1000C30080FBE599227A2879FA78B8D8FED9FADA4A
:1000D300F62275BD0075BF0075BE3075BD037598FA
:1000E30052759100759200224384015385FE43911A
:1000F3008053927FD2C275A12075A303758E05E547
:100103008E30E3FB223031323334353637383941E0
:10011300424344454674301200B874781200B890D4
:100123000108E5F0C4540F931200B8E5F0540F939F
:100133001200B874201200B822E49360061200B8CB
:10014300A380F622D206D205D204D203D202D20170
:10015300D200C3E5C694C44003C20622C3E5C694D5
:10016300AF4003C20522C3E5C694904003C20422F4
:10017300C3E5C694714003C20322C3E5C69452404B
:1001830003C20222C3E5C694334003C20122C3E57E
:10019300C694144003C2002222C0E074011412006A
:1001A3009BD0E07430A20634001200517430A205D3
:1001B30034001200517430A2043400120051743020
:1001C300A20334001200517430A202340012005111
:1001D3007430A20134001200517430A200340012B2
:1001E3000051224144433020707573682062757456
:1001F300746F6E73000D0A41444330207075736849
:1002030020627574746F6E732E202054686520709D
:1002130075736820627574746F6E7320766F6C7477
:100223006167652064697669646572206973206318
:100233006F6E6E656374656420746F2050312E3762
:100243000D0A0075817F75840075850075910075B1
:10025300920075A40075A50075B10075B200120077
:10026300D51200EB12005BC0E074011412009DD0A4
:10027300E0C083C082C0E09001E6120090D0E0D0DD
:1002830082D0831200C89001F812013C740D120051
:10029300B885C5F012011885C6F01201181201477E
:0502A30012019C80E740
:00000001FF
